:0200000480007A
:1000000097170000938707007310003473D10034F2
:100010007352003473D30F3473DE0734735F0834C4
:10002000F35F003423A0070023A2270023A4470086
:1000300023A6670023A8C70123AAE70123ACF70181
:10004000971000009380C0FD73D0073473500034C4
:1000500023A00000171500001305C5FA971500002E
:10006000938545FC370610F01306C6F26306B50209
:100070008326C5002320D600832685002320D600B2
:10008000832645002320D600832605002320D600A2
:10009000130505016FF09FFD370510F0130505F2FC
:0400A0002320050014
:10100000FFFFFFFFFFFFFFFFFFFFFFFFFFFFFFFFF0
:10101000FFFFFFFFFFFFFFFFFFFFFFFFFFFFFFFFE0
:040000058000000077
:00000001FF
